:0200000480007A
:100000006F000005732F2034930F80006308FF03F7
:10001000930F90006304FF03930FB0006300FF038E
:10002000130F000063040F0067000F00732F2034CC
:1000300063540F006F00400093E19153171F0000BD
:1000400023223FFC171F000023200FFC6FF01FFF2F
:100050009300000013010000930100001302000050
:100060009302000013030000930300001304000038
:100070009304000013050000930500001306000020
:100080009306000013070000930700001308000008
:10009000930800001309000093090000130A0000F0
:1000A000930A0000130B0000930B0000130C0000D8
:1000B000930C0000130D0000930D0000130E0000C0
:1000C000930E0000130F0000930F0000732540F102
:1000D0006310050097020000938202017390523072
:1000E000735044749702000093820201739052305F
:1000F00073500018970200009382020273905230EE
:10010000B70200809382F2FF7390023B9302F001EA
:100110007390023A7350403097020000938242017C
:100120007390523073502030735030309301000080
:1001300097020000938242ED739052301305100035
:100140001315F501634C05000F00F00F930110002B
:100150009308D0051305000073000000930200000F
:10016000638A020073905210B7B20000938292101B
:100170007390223073500030372500007320053013
:100180007350300097020000938242017390123442
:10019000732540F1730020309301200017250000E3
:1001A000130545E68316050013052000537005D49A
:1001B00073101000530500E46316D50A9301300054
:1001C00017250000130525E4831605001305E0FF3D
:1001D000537005D473101000530500E46314D50860
:1001E0009301400017250000130505E28316050062
:1001F00013052000537015D473101000530500E44C
:100200006312D50693015000172500001305E5DFA2
:10021000831605001305E0FF537015D4731010000A
:10022000530500E46310D5049301A00017250000D6
:100230001305C5DD071005008710250007114500CF
:1002400083166500D3012040D3F10144538501E4B6
:10025000F3151000130600006316D5006394C50063
:10026000631030020F00F00F6380010093911100C2
:1002700093E111009308D00513850100730000007D
:100280000F00F00F930110009308D0051305000034
:1002900073000000731000C00000000000000000A8
:1002A000000000000000000000000000000000004E
:0C02B00000000000000000000000000042
:1010000000000000000000000000000000000000E0
:1010100000000000000000000000000000000000D0
:1010200000000000000000000000000000000000C0
:1010300000000000000000000000000000000000B0
:081040000000000000000000A8
:10200000004000C00040007C00BE0000000000BE98
:040000058000000077
:00000001FF
